:100000009328003803198E2894000C0884000D18DA
:1000100083178C018D01941B152800088C00941CFB
:100020008E28840A00088D008E2830200005031DCC
:100030008C0A8E28A4008417800484138E010C1C63
:100040008E0024088E0601308C008D0100082405E6
:100050000E06031D08008C0A03198D0F26280800C0
:1000600000308A001408073982070134023404344E
:10007000083410342034403480348F018E00FF3037
:100080008E07031C8F07031C8E2803308D00DF3082
:100090004B203F288D01E83E8C008D09FC30031C6D
:1000A00054288C07031851288C0764008D0F5128A1
:1000B0000C185A288C1C5E2800005E2808008E0050
:1000C0000130622894000F080D02031D69280E08F4
:1000D0000C02043003180130031902301405031D0B
:1000E000FF308E2810309200910190010D0D900D7F
:1000F000910D0E0890020F08031C0F0F91020318B8
:1001000088280E0890070F0803180F0F9107031097
:100110008C0D8D0D920B76280C088E2883130313FB
:100120008312640008008316403086000730850083
:100130008312AC01AD01861783168613013083123A
:100140003D2001308C000630840080301A200C08DD
:10015000AA000D08AB002A088C002B088D000B307C
:100160008F00B8305F20031D3629AE0164000630D1
:100170002E02031835292E088E00053C031CE628A4
:1001800003100E0D8E07D0208C008E0AD0208D001B
:100190008E0AD02001200C08A8000D08A900E6282E
:1001A00000308A000E0882072134103400342234D3
:1001B00002340034A434003400340C3408340034E5
:1001C000143402340034A434003400343F302805A1
:1001D000860028088C0029088D0040308E008F0191
:1001E0007220B10007300505B00030088E00073CD2
:1001F000031C262903100E0D8E070A218C008E0A7F
:100200000A218D008E0A0A2101200C08AC000D087D
:10021000AD00262901308A000E08820764340034BC
:100220000034FA3400340034F43401340034E83457
:1002300003340034D03407340034A0340F34003495
:1002400040341F34003480343E3400340130AF0079
:1002500064002F083102031C33292D088F002C085D
:100260003E20AF0F2829AE0FB6289B28AE016400B0
:1002700002302E0203188B292E08013C031C4A2948
:100280004421A800A9014A2901308A002E088207CA
:10029000023410343F302805860007300505B000D1
:1002A00030088E00073C031C812903100E0D8E07B9
:1002B00065218C008E0A65218D008E0A6521012042
:1002C0000C08AC000D08AD00812901308A000E0831
:1002D0008207643400340034FA3400340034F434D7
:1002E00001340034E83403340034D03407340034AB
:1002F000A0340F34003440341F34003480343E3492
:1003000000342D088F002C083E202D088F002C086B
:0C0310003E20AE0F37299B2863008C298B
:02400E00F53F7C
:00000001FF
